:0200000480007A
:100000006F00C004732F2034930F8000630AFF0336
:10001000930F90006306FF03930FB0006302FF038A
:10002000170F0080130F0FFE63040F0067000F000F
:10003000732F203463540F006F00400093E19153FD
:10004000171F000023203FFC6FF09FFF930000006C
:10005000130100009301000013020000930200004E
:100060001303000093030000130400009304000036
:10007000130500009305000013060000930600001E
:100080001307000093070000130800009308000006
:100090001309000093090000130A0000930A0000EE
:1000A000130B0000930B0000130C0000930C0000D6
:1000B000130D0000930D0000130E0000930E0000BE
:1000C000130F0000930F0000732540F1631005002B
:1000D000970200009382020173905230735000180F
:1000E000970200009382020273905230B7020080A0
:1000F0009382F2FF7390023B9302F0017390023AF5
:100100007350403097020000938242017390523046
:10011000735020307350303093010000970200007C
:10012000938282EE73905230130510001315F5017F
:10013000634C05000F00F00F930110009308D005E9
:10014000130500007300000097020080938282EB89
:10015000638A020073905210B7B20000938292102B
:100160007390223073500030372500007320053023
:100170007350300097020000938242017390123452
:10018000732540F17300203073D030003715000024
:1001900013054523F3153500930310009301200048
:1001A000639C752673253000930340039301300050
:1001B00063147526732510009303400193014000DA
:1001C000631C7524735521009303100093015000A4
:1001D0006314752473253000930340059301600078
:1001E000631C752273751200930340019301700024
:1001F000631475227325300093030005930180007A
:10020000631C7520B755341293858567130600006B
:10021000D38005F0530106F053802020530500E001
:10022000B7533412938383679301A0006316751E3E
:10023000B7553412938585671306F0FFD38005F018
:10024000530106F053802020530500E0B753349249
:10025000938383679301B0006310751CB755349284
:100260009385856713060000D38005F0530106F0DF
:1002700053802020530500E0B753341293838367E3
:100280009301C000631A7518B7553492938585673A
:100290001306F0FFD38005F0530106F053802020B1
:1002A000530500E0B7533492938383679301D000E2
:1002B00063147516B75534129385856713060000CD
:1002C000D38005F0530106F053902020530500E041
:1002D000B75334929383836793014001631E751271
:1002E000B7553412938585671306F0FFD38005F068
:1002F000530106F053902020530500E0B753341209
:10030000938383679301500163187510B755349236
:100310009385856713060000D38005F0530106F02E
:1003200053902020530500E0B753349293838367A2
:10033000930160016312750EB755349293858567FA
:100340001306F0FFD38005F0530106F053902020F0
:10035000530500E0B7533412938383679301700110
:10036000631C750AB7553412938585671306000020
:10037000D38005F0530106F053A02020530500E080
:10038000B7533412938383679301E00163167508B2
:10039000B7553412938585671306F0FFD38005F0B7
:1003A000530106F053A02020530500E0B7533492C8
:1003B000938383679301F00163107506B7553492F8
:1003C0009385856713060000D38005F0530106F07E
:1003D00053A02020530500E0B753349293838367E2
:1003E00093010002631A7502B755349293858567AD
:1003F0001306F0FFD38005F0530106F053A0202030
:10040000530500E0B75334129383836793011002BE
:1004100063147500631030020F00F00F6380010059
:100420009391110093E111009308D0051385010009
:10043000730000000F00F00F930110009308D00527
:100440001305000073000000731000C000000000DE
:10045000000000000000000000000000000000009C
:10046000000000000000000000000000000000008C
:10047000000000000000000000000000000000007C
:040480000000000078
:1010000000000000000000000000000000000000E0
:1010100000000000000000000000000000000000D0
:1010200000000000000000000000000000000000C0
:1010300000000000000000000000000000000000B0
:081040000000000000000000A8
:040000058000000077
:00000001FF
